:107000000C941A390C94FB390C942C390C942C39AF
:107010000C942C390C942C390C942C390C942C395C
:107020000C942C390C942C390C942C390C942C394C
:107030000C942C390C942C390C942C390C942C393C
:107040000C94E3390C942C390C943E3E0C946C3E19
:107050000C942C390C942C390C942C390C942C391C
:107060000C942C390C942C392E007061676553698F
:107070007A6520616E6420626C6F636B506F732061
:107080006469666665720A00546F206D616E7920CE
:107090006461746120666F72207061676553697AFC
:1070A000650A00626C6F636B4C656E20646966668E
:1070B0006572207061676553697A650A0057726F5F
:1070C0006E67204D73674964210A005265747261CE
:1070D0006E736D69742C207265666C617368210A29
:1070E00000476F74206F74686572206D7367547900
:1070F00070650A0052656365697665206669726D20
:10710000776172650A00476F74204342206D736790
:107110000A005761697420666F72204342206D73C4
:10712000670A00545820626F6F746C6F61646572F7
:107130002073657175656E63650A0054696D656FCE
:1071400075740A005374617274204170700A0042B1
:107150006F6F746C6F616465722073656C665570D7
:1071600064617465210A00435243206661696C2C96
:10717000205265626F6F740A00435243204F4B0ADE
:107180000070616765416464722065786365656459
:107190007320666C617368206D656D6F72790A008B
:1071A00053776974636820746F203130306B206DC1
:1071B0006F64650A000A41736B53696E204F544136
:1071C00020426F6F746C6F616465722056302E3789
:1071D0002E300A0A0053776974636820746F203177
:1071E000306B206D6F64650A00002E012E020603CD
:1071F0000D04E905CA063D070C0B060D210E650FAF
:107200005010C811931203153416011730181819AD
:10721000161B432156250026112D353EC30B0810A1
:107220005B11F81547191D1A1C1BC71C001DB22144
:10723000B623EA0011241FBECFEFD8E0DEBFCDBFDA
:1072400011E0A0E0B1E001C01D92A13DB107E1F75E
:107250000E94733C0C940E3F0C9400382FB7F894A6
:1072600085B7982F916095BF826085BF2FBF85B588
:10727000826085BD16BCEEE6F0E08081816080838F
:1072800081E08DBB82E0809369000895CF93DF9306
:10729000809100018823D9F1F89410920001409167
:1072A0009501409359018091960196E78927809333
:1072B0005A01E6E9F1E0CBE5D1E0A1E5B1E030E04B
:1072C00022E013C090819452818198279883822F65
:1072D0008750833030F48C91981711F030E007C05C
:1072E00031E02F5F319621961196241758F3A22F83
:1072F000B0E0FD01EB56FE4F808190915B01892744
:10730000A75ABE4F8C937894832F311181E0DF917F
:10731000CF91089590E041E250E19B01220F331F8D
:1073200087FD216077FD02C0B90103C0B901642760
:1073300075279F5F983011F0880FEFCFCB0108952C
:10734000CF93DF936FEF7FEFC0E0D0E0FE01849139
:107350000E948A39BC012196FFE6CE3FDF07B1F7D4
:1073600080E00E948A39BC0180E00E948A39FE01D7
:107370002591349140E02817390709F441E0842F22
:10738000DF91CF91089550E0A0EDB7E019C05C9A6D
:1073900020E030E005C0FD013197F1F72F5F3F4F4E
:1073A00028173907C0F35C9820E030E005C0FD01E4
:1073B0003197F1F72F5F3F4F26173707C0F35F5F15
:1073C000541728F308951F920F920FB60F921124AD
:1073D0008F939F9316BC80910101909102010196B9
:1073E00090930201809301019F918F910F900FBEA6
:1073F0000F901F9018951F920F920FB60F921124A5
:107400002F933F934F935F936F937F938F939F93AC
:10741000AF93BF93EF93FF93F89485E991E00E94B7
:107420005A3D882319F081E0809300017894FF9100
:10743000EF91BF91AF919F918F917F916F915F91EC
:107440004F913F912F910F900FBE0F901F90189565
:10745000ECEFFFE6859194918151974489F48FE494
:1074600091E70E94EE3E80E09AEF0197F1F782E308
:1074700090E062E370E04AE00E94C3390E94803FDE
:1074800084E491E70E94EE3E80E09AEF0197F1F7E5
:107490005C98F89485B7982F916095BF8D7F85BFD4
:1074A000E0E0F0E0099508950E94A039882329F0D2
:1074B00089E791E70E94EE3E089580ED97E061E054
:1074C00070E041E00E94C33987E691E70E94EE3EFA
:1074D000A8952EE088E190E00FB6F894A8958093E7
:1074E00060000FBE20936000FFCF8091010190915A
:1074F00002018153954740F08BE391E70E94EE3EF5
:107500000E94543A0E94283A08951F93CF93DF9324
:10751000DA0161382FE6720720E0820720E0920747
:1075200028F081E891E70E94EE3E30C0F894F99986
:10753000FECFAB0183E0FB0180935700E89507B6CF
:1075400000FCFDCFFA0111E0BA0160587F4F8C9129
:1075500011963C91119720E0E901C80FD11D1296B8
:107560000E0110935700E89511243296E617F7079D
:1075700071F785E0FA0180935700E89507B600FCA3
:10758000FDCF81E180935700E8957894DF91CF910A
:107590001F910895DC0111969C91119786E7982719
:1075A00011969C93119712965C91129742E008C035
:1075B000FD01E20FF31F94528081982790834F5F63
:1075C0008C91242F30E0481798F3FD01E20FF31F50
:1075D000808185278083F894CD0160E00E94993DE9
:1075E000789408950F931F93DF93CF93CDB7DEB7B1
:1075F00065970FB6F894DEBF0FBECDBF83E291E76B
:107600000E94EE3E90915601209157013091580111
:10761000409148015091490160914A0170914B019C
:10762000E0914C01F0914D01A0914E01B0914F01BC
:10763000109150010091510184E189831A821B82CB
:1076400080E18C839D832E833F83188619861A865A
:107650001B864C875D876E877F87E88BF98BAA8BAB
:10766000BB8B1C8B0D8BCE0101960E94CA3A65968E
:107670000FB6F894DEBF0FBECDBFCF91DF911F9143
:107680000F910895DF93CF93CDB7DEB72B970FB649
:10769000F894DEBF0FBECDBFFC01A62F662319F400
:1076A000828185FF1CC09181209156013091570144
:1076B000409158015481658176818AE089839A835B
:1076C00080E88B8382E08C832D833E834F835887B1
:1076D00069877A87AB87CE0101960E94CA3A2B96BA
:1076E0000FB6F894DEBF0FBECDBFCF91DF910895E6
:1076F0002F923F924F925F926F927F928F929F92C2
:10770000AF92BF92CF92DF92EF92FF920F931F93AF
:10771000DF93CF93CDB7DEB7C058D0400FB6F89403
:10772000DEBF0FBECDBFA0905A0110920201109291
:10773000010184EF90E70E94EE3EBB2400E010E0E0
:10774000CC24DD2476012E010894411C511C83E6D3
:10775000682E81E0782EB2E02B2E312C260C371CBF
:1077600002C0BB24B3940E94753A0E944639882314
:10777000D1F380915C018A3C19F081EE90E731C031
:1077800080915A018A1581F4BB2071F4C114D1048F
:10779000E104F10449F00894C108D108E108F108B6
:1077A0008BEC90E70E94EE3E80915A018A1550F4CE
:1077B00025E72A1520F48A2D8158843718F48DEB9B
:1077C00090E748C0BB20E1F4909063018824809149
:1077D00064019401280F311D2038310529F083EA16
:1077E00090E70E94EE3EBFCF80915901082F10E034
:1077F0000B501040C201B101A8010E94053F20C0FA
:1078000080915901E82FF0E03997CF01800F911F47
:107810008138910518F088E890E71CC09201200F8C
:10782000311FC901B301AF010E94053F8091590189
:1078300090E00997080F191F31E0B31609F093CFB4
:1078400080915B01803209F08CCF0038110529F05E
:107850008AE690E70E94EE3E22C088E690E70E940A
:10786000EE3E5C9AC701B601A7E0660F771F881F3E
:10787000991FAA95D1F7A2010E94853A0894C11CCC
:10788000D11CE11CF11C10920201109201015C98C4
:10789000A0905A0189E591E060E00E94423BBB2440
:1078A00062CF82E191E70E94EE3E109202011092B7
:1078B00001010E94753A0E9446398823D1F38091D4
:1078C0005C018B3C51F486E091E70E94EE3E89E535
:1078D00091E060E00E94423B089589E591E060E814
:1078E0000E94423BE6CF1F9314B716951695169546
:1078F000117014BEA89588E10FB6F89480936000CB
:10790000109260000FBE2098289A8AE18A95F1F7BC
:10791000549A189B33C0112389F58CE291E06CE2F4
:1079200071E040E00E94C33988E893E128EC30E040
:10793000F9013197F1F70197D9F786E990E066E907
:1079400070E047E00E94C33988E893E128EC30E01A
:10795000F9013197F1F70197D9F78CE291E06CE2E8
:1079600071E040E00E94C33980E197E228EC30E00A
:10797000F9013197F1F70197D9F707C089E190E054
:1079800068EC70E041E00E94C3390E942E3985ED19
:1079900091E70E94EE3E80E00E94DC3D88E090E0AE
:1079A0000E94963E85EB91E70E94EE3E189B08C030
:1079B000112331F40E94A039882311F00E94283A43
:1079C00089E190E068EC70E041E00E94C33986E50F
:1079D00091E06CEF7FE743E050E00E94FC3E88E4DA
:1079E00091E062EF7FE74AE050E00E94FC3E0E9497
:1079F000F23A0E94513C80EA91E70E94EE3E81E01B
:107A00000E94DC3D0E94513C0E94783B80E090E067
:107A10001F9108958EBD0DB407FEFDCF8EB508955C
:107A20002A982C99FECF8EBD0DB407FEFDCF8EB5E2
:107A30002A9A08952A982C99FECF80648EBD0DB4A1
:107A400007FEFDCF8EB5FB0190E008C080818EBDA2
:107A50000DB407FEFDCF8EB59F5F31969417B0F33E
:107A60002A9A08959C012A982C99FECF606C6EBDCD
:107A70000DB407FEFDCF8EB5F90190E007C01EBC26
:107A80000DB407FEFDCF8EB581939F5F9417B8F3B9
:107A90002A9A08952A982C99FECF682B6EBD0DB4B2
:107AA00007FEFDCF8EB51EBC0DB407FEFDCF8EB513
:107AB0002A9A0895CF93DF93EC018BE360EC0E9448
:107AC0004A3D282F90E08F779070892B09F127FD90
:107AD0001FC08FE360E80E944A3D482F88838D33A2
:107AE000B8F4CE0101966FE30E94323D8FE360E867
:107AF0000E944A3D8FE360E80E944A3D982F9F779D
:107B000090935501881F8827881F8093530101C0D7
:107B100018828AE30E94103D86E30E94103D84E3B0
:107B20000E94103D8CE30E94103D8881DF91CF912F
:107B300008950F931F938C0186E30E94103D8AE302
:107B40000E94103D8BE30E94103D80ED97E001976D
:107B5000F1F7F80140814F5F8FE3B8010E941A3DB1
:107B60008AE30E94103D85E30E94103D00E01AE187
:107B700085E360EC0E944A3D8D3061F085E360EC66
:107B80000E944A3D833131F4812F8A95F1F70F5FCE
:107B9000083C71F71F910F9108952A982C99FECFF8
:107BA0008EBD0DB407FEFDCF8EB56EBD0DB407FEC4
:107BB000FDCF8EB52A9A08951F93CF93DF93182F88
:107BC000F894229A239A2498259A52982A9A2D9AC0
:107BD0002B9880E58CBD2A9A982F9A95F1F72A98D0
:107BE0008A95F1F72A9A88E78A95F1F780E30E944F
:107BF000103D88EC90E00197F1F7C9EED1E7FE0166
:107C000084912196FE0164910E94CD3D2196F2E778
:107C1000CD31DF07A1F7112371F0CDE1D2E7FE01ED
:107C200084912196FE0164910E94CD3D2196F2E758
:107C3000C333DF07A1F783E30E94103D80E49FE197
:107C40000197F1F784E30E94103D85E360EC0E9408
:107C50004A3D8D30B9F78EE360EC0E94CD3D84E360
:107C60000E94103D8CE30E94103D80E797E1019750
:107C7000F1F77894DF91CF911F9108951F920F92A1
:107C80000FB60F9211242F938F939F93EF93FF932F
:107C90009091C0002091C600E0914501EF5FEF7127
:107CA00080914601E81711F492E007C09871E093C3
:107CB0004501F0E0ED5DFE4F208380914701982B58
:107CC00090934701FF91EF919F918F912F910F908A
:107CD0000FBE0F901F9018951F920F920FB60F9224
:107CE00011248F939F93EF93FF9390914301809181
:107CF0004401981769F0E0914401EF5FEF71E09360
:107D00004401F0E0ED5FFE4F80818093C60005C026
:107D10008091C1008F7D8093C100FF91EF919F9171
:107D20008F910F900FBE0F901F9018959C0110928D
:107D3000430110924401109245011092460197FFB1
:107D400004C082E08093C0003F773093C500209349
:107D5000C40088E98093C10086E08093C200089542
:107D60009091450180914601981719F420E031E087
:107D700010C0E0914601EF5FEF71E0934601F0E043
:107D8000ED5DFE4F80819091470110924701282FB1
:107D900030E0C9010895282F909143019F5F9F71A2
:107DA000809144019817E1F3E92FF0E0ED5FFE4F79
:107DB0002083909343018091C10080628093C10031
:107DC0000895CF93DF93EC0103C021960E94CB3E30
:107DD00088818823D1F7DF91CF910895CF93DF93E6
:107DE000EC0102C00E94CB3EFE01219684918823C3
:107DF000C9F7DF91CF910895FB01DC0102C0059026
:107E00000D9241505040D8F70895FB01DC0102C0AB
:107E100001900D9241505040D8F70895F894FFCF4B
:107F0000FF920F931F93CF93DF93F8945C9AC0E096
:107F1000D0E7F3E0FF2E01E015E0FE01F0925700FC
:107F2000E89507B600FCFDCFAE0140505047BE01BA
:107F3000DE01A058BF46FA0185919491FB010C0126
:107F400000935700E89511244E5F5F4F6E5F7F4F9F
:107F50004A175B0781F7FE0110935700E89507B6B3
:107F600000FCFDCFC058DF4FFFE7C030DF07A9F6A8
:107F7000E0E8FFE683E080935700E89507B600FC51
:107F8000FDCF81E180935700E8955C982EE088E171
:107F900090E00FB6F894A895809360000FBE2093F0
:047FA0006000FFCFAF
:027FF000123449
:0A7FF20048423044656661756C7406
:037FFC00ABCDEF1B
:040000030000700089
:00000001FF
